:020000040800F2
:1040000058080020654100087552000879520008E0
:104010007D5200088152000885520008000000000F
:104020000000000000000000000000008D520008A9
:1040300089520008000000009152000895520008C3
:10404000995200089D520008A1520008A55200088C
:10405000A9520008AD520008B1520008B55200083C
:10406000B9520008BD520008C1520008C5520008EC
:10407000C9520008CD520008D1520008D55200089C
:10408000D9520008DD520008E1520008E55200084C
:10409000E9520008ED520008F1520008F5520008FC
:1040A000F9520008FD5200080153000805530008AA
:1040B000095300080D530008C5530008C9530008F0
:1040C000CD530008D1530008D5530008D953000838
:1040D000DD530008E1530008E5530008E9530008E8
:1040E000ED530008F1530008F5530008F953000898
:1040F000FD53000801540008055400080954000845
:104100000D540008115400081554000819540008F3
:104110001D540008215400082554000829540008A3
:104120002D54000831540008355400083954000853
:104130000120704710B5094C02E004F0A3FB0C34D9
:104140000748844208D26068A16822688142F4D19D
:10415000002104F0A3FBF2E710BD00BF3C8900087A
:1041600054890008024CA04730B1024CA04703E03C
:104170003141000835410008034C4FF00000A047D2
:10418000024C034DAE4620474D5B000825880008D1
:044190001989000881
:1042000004F0C0B902F0D8B801F018B901F016BB3B
:1042100053E052E001F04EBB01F064BB01F036BC4C
:1042200058E057E073E072E07BE07AE048E047E076
:104230005AE059E085E057E000F066BF3AE039E027
:1042400032E031E033E032E001F058BB00F09AB8E0
:1042500000F0CABA00F0DABA01F05ABE01F082BE2C
:1042600001F02ABE01F0A6BE01F0C4BA04F08CB879
:1042700000F0E6BF00F0CEBF03F002BB03F008BBC6
:1042800000F00AB800F00CB802F080BB02F048BFA2
:1042900003F062B903F07EB8304B00201B6818476A
:1042A0002F4B00201B6818472E4B1B6818472E4BBE
:1042B0001B6818472D4B1B6818472D49088070470D
:1042C0002C49C869012240EA0200C861086A002836
:1042D000FCD1704728498868012240EA02008860C2
:1042E000C8680028FCD17047224B47F2C152DA61FE
:1042F0001A6A002AFCD147F2C052DA6140F2C902C0
:104300001A625862996247F2C152DA6170471A4BD9
:1043100045F290529A605861D96045F291529A6084
:104320007047154B45F211529A60DA68002AFCD1A9
:1043300045F210529A605861D96045F211529A6064
:1043400070470E4940F220020D4B4A6118884FEA2F
:1043500000400A6119880844704700002C000008DA
:104360003800000828000008240000082000000889
:104370000000006000000240000402400010014004
:1043800000000064C74AC84B2DE9F04F81B08DF89A
:1043900000000820804610208146C4485FF4804613
:1043A000B3469DF800600C00C149450CAA46C14DBA
:1043B000272E00F2BB81DFE816F0280039004A0002
:1043C0004D005200590060006F0071008900960096
:1043D0009000E900300141014301460153015501BC
:1043E00064016701B901B901B901B901B901B901A4
:1043F000B901B901B901B9017F01A801A801AC0156
:10440000B901A801A801A801A801CA48B4F5803FD4
:1044100007D2C9495FF4EB720A60D4F5E17101601B
:1044200084E1C549220C0A60A1B2F8E7C348B4F59B
:10443000803F07D2C0495FF4EB720A60D4F5E171A6
:10444000016073E1BC49220C0A60A1B2E7E7BC48F5
:1044500004606BE1BB486421B1EB5401DFE7BA486B
:1044600001222240016851EA8251E9E7002C14BF81
:10447000C3F80080C2F8008058E1012C04D1B34990
:1044800002200860286051E1002C40F04F81C3F801
:104490000090C2F8009049E1AD48D9E7AD48AE4977
:1044A00024B900220260AD4808603FE1012C03D12D
:1044B00000220260AA48F7E7AA4A0A60032140F8EE
:1044C0000C1B40F8084B641C6108A8E7012C19BFBD
:1044D000012101600120086028E12022012C14BF85
:1044E00002600A6022E10422430D082C00F21E81C2
:1044F000DFE814F009001100190021002900300044
:1045000037003E0045009149C0F800900B60026002
:10451000C0F800800AE18D4CC0F8009023600A606A
:10452000C0F8008002E1894CC0F80090236002606E
:10453000C1F80080FAE0C0F80090844803600A6087
:10454000C1F80080F2E0C1F800902B600260C0F872
:104550000080EBE0C1F800902B600A60C0F800809A
:10456000E4E0C1F800902B600260C1F80080DDE05B
:10457000C1F800902B600A60C1F80080D6E0C0F856
:1045800000902B600A60C1F80080CFE05FF4004526
:104590004026082C00F2CA80DFE804F0050C12194E
:1045A0001F252C323900C3F800A00660C3F800B004
:1045B0001D60BBE0C3F800A00660C2F800B0F7E7DA
:1045C000C3F800A00660C3F800B01560AEE0C3F801
:1045D00000A00660C2F800B0F7E7C2F800A00E60C5
:1045E000C3F800B0E4E7C2F800A00E60C2F800B063
:1045F0001D609BE0C2F800A00E60C3F800B0E4E7C5
:10460000C2F800A00E60C2F800B015608EE0C3F8DA
:1046100000A00E60C2F800B0D7E7534853490160CC
:104620005348802101605348534901605348012198
:1046300001605348852140F82C49F0E6514807E7CE
:104640005148046072E0514804604A48016851F4DE
:10465000802101604E488421016048480021DEE647
:104660004C48F5E640487FF0706201680A400260FD
:10467000016851F0306101604748812140F83449B8
:10468000CDE646480021DBE64548012C04D14549EA
:10469000C1F800A08421C2E64349C1F800A08521E9
:1046A000016043E014100140101001401018014057
:1046B00014180140140C01403C4C7FF070612068DC
:1046C000260D01402160206850F080702060C5F800
:1046D00000B0012001F0AAF81C480660012001F09A
:1046E000A5F82E60012001F0A1F81848C0F800B02C
:1046F000022001F09BF820687FF07061014021608A
:10470000206850F00060206010E09DF80000E1B2E9
:104710000AE09DF80000E1B200F066F89DF80000A4
:10472000210AC9B2401CC0B200F05EF8002001B0FE
:10473000BDE8F08F340C00402C0C0040380C0040D9
:104740003434014038340140083C0140100C014031
:10475000282C0140202C01400410024002841D043A
:1047600002841D0702841D00000C014038B4BB34D4
:104770000008004000080140BB1110110074004007
:104780002C14004050040240480402402808004015
:10479000001400402C080040340800401004004081
:1047A000002C01401414014010140140040C01407D
:1047B0000B490C4B70B440220A600025802406008F
:1047C000AE40360654BF1C600C601A600A606D1C57
:1047D000EDB2082DF3D31C601A600C6070BC7047FA
:1047E000100801401408014030B5C0060C0006490D
:1047F0002025C00E0D60FFF7DBFF75480560200027
:10480000BDE83040D4E7000010100140674A684B13
:104810002DE9F041674D0C00674998466C4B202606
:10482000102800F2C080DFE800F009160E1E26579F
:104830005C6365686A6D708A779AA5005FF0C8400E
:104840001E600088B0E05FF0C8401E600088042150
:1048500001408810A8E05FF0C8401E600088102169
:1048600001400811A0E05FF0C8401E6000880821E8
:104870000140C81098E0514873020268050D1340CA
:104880004F4A14682540146853EAC503450D254076
:10489000146853EA5503850D2540046853EA45031F
:1048A000450C25401468126853EAD503850C254051
:1048B000C40C144053EA550353EA44020368B0029F
:1048C000402518400B68104308221A40024308682C
:1048D00005401543280067E0086804210140880866
:1048E00062E038485FF4AF6100684843800A5BE0EB
:1048F0003835EFE7EC35280056E01C35EAE705F2DD
:10490000083051E01068C00B4EE010680121000A29
:10491000014091F0010047E0FFF7B2FC08B91435FF
:104920002800002C40D0017883786422C0780A24C3
:10493000634301FB023108184146401834E0FFF799
:10494000A1FC08B90D352800002C2DD00178837802
:104950006422C0780A24634301FB0231EBE71A4862
:1049600014B3017883786422C0780A24634301FB7E
:104970000231E0E71E60154E5FF0C84000888509EF
:104980002900300000F0C4FAB07830702E2070702A
:10499000F078B0703079F07000203071002C14BFC6
:1049A0002846304600E00020BDE8F081080C0140B8
:1049B00030EBFFFF888A0008081401400808014016
:1049C000081001404C3C0140AC9500083401002027
:1049D0001410014010B5184C03F036F85FF4803025
:1049E00003F052F803F06EF82070012817D1102060
:1049F00002F03AFF022002F02DFF1048104901603A
:104A0000012003F077F8392003F090F80028FAD05D
:104A1000022003F075F803F07BF80828FBD1094861
:104A2000094940F8041B09490160002003F076F8A9
:104A300007480849016010BD5204002004100240DC
:104A400002841D0014100240170100007DAE00001A
:104A50001C1002402F80802030B581B05FF480416F
:104A6000480302F0E5FF5FF4C06002F097FF1420F6
:104A70008DF8000001208DF801008DF802008DF8FE
:104A80000300684602F092FF012413208DF8000015
:104A900020468DF8010000258DF802508DF80300A6
:104AA000684602F083FF1D208DF8000020008DF87D
:104AB00001008DF802508DF80340684602F076FF41
:104AC00001B030BD18481949194A40F8041B19496A
:104AD00040F8081B184901601848194940F8041BA0
:104AE00023490160174918480860184941F8042B08
:104AF000174A41F8082B174A0A601749174A41F824
:104B0000042B174A41F8082B164A0860164941F849
:104B1000042B5FF0BB3241F8082B086013485FF0AC
:104B200080610160704700BF00080140BB888011B0
:104B3000001011BBBB3B8388FFE70000000C014065
:104B400018B8BB3B0C0C0140FFFF000000100140F7
:104B500088883833EFFF000000140140BB84BBB8E5
:104B6000BB1B13BB833333B3001801400400014067
:104B70003833888808480949094B5FF020420160B2
:104B800008490948086009491160094A1360094A3F
:104B90001060094801607047040000A0020F101067
:104BA00002071010040100A00104101011500000B1
:104BB0000C0000A00C0100A0080000A010B5114CD2
:104BC00085B00020ADF800005FF48271ADF80210EE
:104BD000ADF804000221ADF806100121ADF808106F
:104BE0004902ADF80A1003900720ADF8100069469D
:104BF000200002F0B9FF0121200002F0CDFF05B036
:104C000010BD00BF003C00401448154940F8081989
:104C10005FF4D55101601349820C0A60016851F0BC
:104C2000010140F8141B104901601048002140F8B0
:104C3000041B5FF0C04140F80819016851F0010100
:104C400001600B4940F8401B242140F8041B09492E
:104C500040F8081908490160704700BF1000024081
:104C60004C2401400C000240C07500000C040240BE
:104C70009175000008740040B1350000034801211F
:104C800040F8081BC10C0160704700BF0074004071
:104C9000304930B4304C0020086030495FF4BC0229
:104CA0005FF480130C2508602D4908602D490A60C7
:104CB0002D4A13602D4B1C602D4C20602D4C206024
:104CC0002D4C20602D4C25602D4C0B2525602D4C46
:104CD0000A2525602C4C802525602C4C20602C4C0E
:104CE0002060086850F001000860106850F0010072
:104CF0001060186850F001001860086850F0080053
:104D0000086008680007FCD4106850F008001060C4
:104D100010680007FCD4186850F008001860186884
:104D20000007FCD4086850F00400086010684007D1
:104D3000FCD4106850F00400106010684007FCD4E8
:104D4000186850F00400186018684007FCD430BCA4
:104D5000704700BF043C01400001100004280140DE
:104D600004240140083C0140082801400824014077
:104D70002C3C01402C2801402C240140343C0140B3
:104D800034280140342401400C3C01400C280140EF
:104D90000C240140354870B4354D092140F8041BFE
:104DA000232140F8081B122140F81419314903222D
:104DB00040F80829782303605FF4004041F838097F
:104DC00000240C60852129602B4D472645F8046B93
:104DD0002A4E2E602A4E012546F80C593160294E84
:104DE0003260294A294E42F8086B294E42F814696C
:104DF000C60942F80859274D1360274B81221A60D3
:104E0000264B43F8044B264C1C60264C5FF49673EB
:104E100044F8043B2360244B33241C60234C244B74
:104E200044F818392260234C13222260632445F889
:104E3000204945F80869082645F8046929601E4993
:104E4000C72541F8045B41F8084B322441F8044B74
:104E5000642441F8184941F8082941F82C3B0860BE
:104E600016489121016070BC704700BF282C01409A
:104E7000002C0140442C014028040040E7030000BE
:104E80000C040040280800402C0800404F46000059
:104E9000282300002C14004000080040280C00408B
:104EA000F3010000340C0040200C0040180C0040BE
:104EB0007878000028140040283401400034014074
:104EC0000F481049104A10B4006809681268A8B168
:104ED0000E4B040A98701C71040C9C71000E187221
:104EE0009972080A1873080C9873080E18749A744B
:104EF000100A1875100C9875100E187610BC7047B3
:104F0000E8F7FF1FECF7FF1FF0F7FF1F000000207E
:104F100002000800154900B590FBF1F3303313701F
:104F200003F006FD80B25FF47A7190FBF1F130314D
:104F300051705FF47A7103F0FBFC80B2642190FB46
:104F4000F1F130319170642103F0F2FC80B20A215A
:104F500090FBF1F13031D1700A2103F0E9FC3030DF
:104F60001071002002F8050F00BD00BF10270000DF
:104F70000A0F0A2A39BF303200F8012B373200F805
:104F8000012B090109090A0E0A2A39BF303200F83B
:104F9000012B373200F8012B0902090A0A0D0A2AEF
:104FA00039BF303200F8012B373200F8012B0903EA
:104FB000090B0A0C0A2A39BF303200F8012B3732AC
:104FC00000F8012B89B20A0B0A2A39BF303200F8E7
:104FD000012B373200F8012B0905090D0A0A0A2AAC
:104FE00039BF303200F8012B373200F8012BC9B23B
:104FF0000A090A2A39BF303200F8012B373200F88B
:10500000012B0907090F0A2939BF303100F8011BAC
:10501000373100F8011B002101707047F0B5002105
:10502000234E04200024FFF7F1FBC143214889B23D
:105030000A00038805259A43170020D019273770E6
:10504000D60548BF0324960548BF0424560548BF2B
:105050000524150548BF0624D30448BF072493043C
:1050600048BF0224530448BF0124130448BF082446
:10507000130748BF0924520616D50A2414E00288F3
:10508000114211D032787AB90B4A167866B94E05BA
:1050900048BF05240E0548BF06240B0748BF092456
:1050A0000B0448BF0824157001802000F0BD00BF2C
:1050B000350400204404002036040020024A1180F8
:1050C00001000320FFF75EB9420400200D4940585B
:1050D0007047000070B506000D0002F0D1FB0948D2
:1050E000B1B2281800F096F804000548310C2818D1
:1050F00000F090F80500254002F0CAFB280070BDC2
:1051000006380008043800082DE9704D87B00024E7
:105110000E003C49804668460A780025B246027077
:105120004A782146427004A8FFF722FF36482346FA
:105130005146834604A801B45A46404600F0DEFBBF
:1051400001B0290004A8FFF713FF30480199027845
:10515000C9B291421CD000780026019004A9895D53
:1051600018EBC600B4428DF80010694602B404D1B1
:10517000029B5A465146DBB202E000235A46514692
:1051800080B200F0BBFB01B0761CF6B2082EE5D36E
:105190001F48017800292FD006780721091B8B00B2
:1051A000012199400F229A4035FA03F3022E20D0B4
:1051B000052E06D0062E09D0082E0ED0092E12D0AC
:1051C00018E01B070CBFAD186D1A13E01B071B0F6F
:1051D0000F2B2CBFAD1A6D180CE0072C2EBF00242E
:1051E000641CE4B206E021000EBF0724641EE4B292
:1051F00000E0082400210170082CA2D3280007B089
:10520000BDE8708D4C960008FFFF00003A040020B6
:105210003704002030B5040015480D0002F09AFB59
:1052200005281CBF342002F07DFB2900200002F07D
:1052300057FB042804BF012030BD002030BD000012
:1052400010B50400600510D1094802F083FB052861
:105250001CBF342002F066FB200002F01FFB042874
:1052600004BF012010BD002010BD012010BD0000B2
:10527000A086010070470000FEE70000FEE7000086
:10528000FEE70000FEE700007047000070470000E6
:105290007047000070470000704700007047000032
:1052A0007047000070470000704700007047000022
:1052B0007047000070470000704700007047000012
:1052C0007047000070470000704700007047000002
:1052D00070470000704700007047000070470000F2
:1052E0007047000003F04EB901F066B87047000047
:1052F00070470000704700007047000070470000D2
:105300007047000070470000704700002A4830B521
:105310002A4D00240460287918B12879401E28718C
:1053200030BD1420287129892548152931BF2C81C9
:10533000298909182981E989152908D3E9890818D3
:10534000E881E889152811D2002103200CE0687952
:10535000322803D26879401C687107E06C71688953
:105360000121401C68810420FFF70CF82878401CBC
:10537000287028780C2809D32C70A87900B901244A
:10538000AC71A88910B1A889401EA881687810B1B5
:105390006878401E6870A87810B1A878401EA87080
:1053A000FFF73CFE010006D0E87014210320FEF751
:1053B000E9FF3C20E88130BD1004004034040020A7
:1053C000ECFF0000704700007047000070470000CD
:1053D00070470000704700007047000070470000F1
:1053E00070470000704700007047000070470000E1
:1053F00070470000704700007047000070470000D1
:1054000070470000704700007047000070470000C0
:1054100070470000704700007047000070470000B0
:1054200070470000704700007047000070470000A0
:105430007047000070470000704700002DE9F04100
:10544000D94DD84F0120AE0C2E60EC0C2C6000F032
:10545000EDF93C600A2000F0E9F92C60322000F000
:10546000E5F900F0A3F9E248BF495FF0C0440068E5
:1054700088426AD1E92000F08BF920202080112099
:1054800000F086F9642000F0D1F9D12000F080F915
:10549000002525805E20208017202080D02000F06D
:1054A00077F90720208020800C202080362000F013
:1054B0006FF940208046A4F800800C2000F068F9C5
:1054C000552626803A2000F063F92680C12000F09E
:1054D0005FF9102020802080022626802680C020B0
:1054E00000F056F925803520208025802580012771
:1054F00027802680C52000F04BF92780D22000F0BD
:1055000047F9278022202080C82000F041F9278019
:10551000732020803720208025800F202080268047
:1055200004212180A4F80080672121802580268025
:10553000208008202080802020802580292000F0E5
:1055400027F92C2000F024F9DCE00021002000F0F5
:1055500013F90021084600F00FF90021084600F079
:105560000BF90021084600F007F90A2000F05EF967
:105570000121200D00F000F90A2000F057F9402128
:105580005FF4DE6000F0F8F80A2000F04FF95FF4F5
:10559000C441280D00F0F0F85B49082000F0ECF859
:1055A000A90D012000F0E8F8A90D022000F0E4F8B0
:1055B0003021032000F0E0F80121092000F0DCF8A0
:1055C00000210C2000F0D8F8F100902000F0D4F871
:1055D00000210F2000F0D0F81621102000F0CCF8A8
:1055E0004A4880464146112000F0C6F800211220AA
:1055F00000F0C2F80121132000F0BEF85FF44C71F6
:10560000A80D00F0B9F84249404600F0B5F841480D
:105610005FF4706100F0B0F85FF4D6415FF4207081
:1056200000F0AAF83C495FF4817000F0A5F864200E
:1056300000F0FCF8E10C880800F09EF83749384883
:1056400000F09AF83749384800F096F8374938485A
:1056500000F092F85FF40C515FF4417000F08CF8A8
:1056600034485FF4B85100F087F83349334800F00C
:1056700083F83349334800F07FF833495FF44270D0
:1056800000F07AF83149324800F076F800215FF4F2
:10569000047000F071F83548EF2100F06DF83448DF
:1056A000002100F069F82B49324800F065F800212C
:1056B0005FF4A06000F060F80021274800F05CF87B
:1056C0002648052100F058F82548012100F054F83B
:1056D0002448002100F050F8642000F0A7F8A90D3C
:1056E000072000F049F8642000F0A0F80021680DC0
:1056F00000F042F86D48002100F03EF86C483E6032
:1057000020802E60BDE8F081080800000101000043
:105710003702000003010000B0C100000B5A000076
:10572000010300000609000002030000171000003A
:1057300003030000050300000963000006030000E6
:10574000090C0000070300000C10000032220000CA
:10575000090300008F0100000105000002050000A0
:105760000104000004040000279304021102000059
:1057700012020000130200000A4B5FF480521A600C
:105780005FF0C0431880084802601980704700002D
:10579000044A5FF4805111605FF0C04210800248FB
:1057A00001607047141401401014014000B5EF204F
:1057B000FFF7EEFF5FF0C04000880D485FF0C0418A
:1057C00009885FF0C042090601601288D2B251EA2E
:1057D00002415FF0C04201601288D2B251EA022158
:1057E0005FF0C04201601288D2B20A43026000BD7D
:1057F0003C010020CC48CD4910B5006888420CD14E
:105800002E20FFF7C5FF5FF0C04000885FF0C0406A
:1058100004882C20FFF7BCFF05E05FF0C040008843
:105820005FF0C0400488200010BD000002490880DD
:1058300008880028FCD170473C04002070B50500A2
:105840005FF0C0440E00FEF7EBFCB748B7490068B4
:10585000884218D12A20FFF79BFF00202080F1B258
:1058600021802080EF2020802B20FFF791FF280A45
:105870002080E8B22080012020808F2020802C20F2
:10588000FFF786FF70BD31005FF40070FFF774FF13
:1058900006482900FFF770FFA9495FF480500860AF
:1058A00003492180A849086070BD00000102000082
:1058B0000202000030B5094C094D00212080002073
:1058C000FFF7BCFF29002000FEF7AEFCFEF7A8FCA6
:1058D00029002000BDE83040FEF7A6BC46040020A9
:1058E00080BB0000034A11EBC000034911EB4000EC
:1058F000805A7047E0FDFFFFD08E00082DE9F04F81
:1059000088461C00060000259146FFF797FF1CB94A
:105910000020FEF77DFC04E0012C04BF4846FEF7A2
:1059200077FC6D1C0E2DF2DB0998761CB3460078CF
:10593000002844D0002641465846801980B2FFF71F
:105940007DFF09980078202801D021280CD100275C
:10595000212801D1042E27D0002578070DD544B980
:105960004846FEF755FC12E0B1B2FFF7BBFF070057
:10597000F2E7012C0BD10020F3E71CB90020FEF761
:1059800047FC04E0012C04BF4846FEF741FC3F04FD
:105990007F146D1C0E2DE0DB761C36B2082ECADBA0
:1059A00009980078212802D10BF2040B01E00BF2D8
:1059B000080B0998401C099000780028BAD1BDE86E
:1059C000F08F00002DE9F04F88B00C0000258046D4
:1059D00081464F46002115E0284B294E0A0013F856
:1059E000223016F822606846DB08B608760116EB0E
:1059F000C323244E491C89B216F82260F6089B196D
:105A000020F812301029E7D330E021003800FFF7EA
:105A100015FF1D497F1CBFB2481982465FF0C04088
:105A200083469AF8000069464646001131F8100096
:105A3000FF36BE42ABF80000BEBF4F46641CA4B2A6
:105A400021003800FFF7FAFE9AF8000069467F1C33
:105A50000007000F31F81000BFB2BE42ABF80000E3
:105A6000BEBF4F46641CA4B26D1CADB25FF40051C2
:105A70008D42CAD308B0BDE8F08F00BF36D8030806
:105A800037D8030838D8030876D803082DE9F04141
:105A90000500254888462549006816001F005FF06C
:105AA000C04488421BD12A20FFF772FE300A2080B2
:105AB000F0B22080380A2080F8B220802B20FFF737
:105AC00067FE280A2080E8B220804046000A208035
:105AD0004046C0B220802C20FFF75AFE21E0144837
:105AE0003900FFF749FE13484146FFF745FE3100F4
:105AF0005FF40470FFF740FE0F482900FFF73CFEFB
:105B000031005FF40070FFF737FE0C482900FFF703
:105B100033FE0B495FF4805008600A4921800A492E
:105B20000860BDE8F08100003C01002027930402DA
:105B30001102000013020000120200000102000026
:105B40001414014002020000101401402DE9F0413C
:105B5000754C764D83B0FEF73DFFFEF77DFFFEF7F7
:105B6000B1FFFFF717F9FFF705F8FFF727F8FFF781
:105B70004BF8FFF78DF8FFF781F85FF4FA71142006
:105B8000FFF79CFAFFF75AFC0020FFF793FE9621DF
:105B90004620FFF717FF10B400235FF4FC625A2180
:105BA0002820FFF7ABFE00210D20FEF72FFE01B4E9
:105BB00000235FF4FC625A219020FFF79FFE200033
:105BC000103001B400235FF4FC625A21C820FFF7B3
:105BD00095FEFEF733FB010003A8FFF7C9F954480F
:105BE00000235A21804603A801B442465FF4907016
:105BF000FFF784FE20001C3001B400235FF4FC6238
:105C000046213020FFF77AFE00210F20FEF7FEFD2F
:105C100001B400235FF4FC6246215FF48870FFF753
:105C20006DFE4448016806B0490554D501688905F0
:105C300051D50168C9054ED53F4E00203070FFF7A1
:105C400045FAFEF7FDFA01283FD02000443001B4A8
:105C500000235FF4FC6232213020FFF74FFE322137
:105C60005FF48C70FFF750FA0700FEF7E9FA01B015
:105C7000012805D020006C3001B40023424612E018
:105C800000213800FFF726FA012806D120009430C1
:105C900001B400235FF4FC6205E02000BC3001B4D5
:105CA00000235FF4FC6232213020FFF727FE01B0B1
:105CB000E43410B400235FF4FC621E213020FFF7AF
:105CC0001DFE01B030780028FCD01C4800686860D8
:105CD00028601B4819E00168490505D41948006887
:105CE00068602860184810E00168890505D41748E5
:105CF000006868602860164807E00068C00507D49F
:105D000014480068686028601348006800F008FEC6
:105D100012481349016002F037FB286880470020D1
:105D200003B0BDE8F08100BFA0940008400100204E
:105D3000FF070000081001403704002004C00008DD
:105D400000C00008044001080040010804C0010828
:105D500000C0010804400208004002080408014095
:105D6000BBBB8B8870B54F4C4F4D22682B7833B935
:105D7000504368615143A9610120287001E0012B63
:105D80002FD14A4E686870B9696992B2300000F04C
:105D9000E9F840229821300002F034FC20684038B5
:105DA000686040200AE0A86840229821301802F07C
:105DB00029FC686840386860A8684030A8604021C5
:105DC000012002F0DFFC3021012002F053FC686961
:105DD00040306861A8694038A86135488168403919
:105DE0008160A86930B9334903226860A86068619E
:105DF0000A70287070BD00002A4AF0B52A4D0026AE
:105E0000EB6812682C78403334B95043E861514351
:105E100029620120287001E0012C32D1234C2E612F
:105E200009E028691D4FE9683F5C401C6754286100
:105E3000E868401CE860E8689842F2D3184FE969C6
:105E400038880B18296AEB61081A2862110002F0E1
:105E500069FD60B9EE60991A200000F059F8E86910
:105E60007FF0FF01411804F2001000F051F81048D3
:105E70003A888168891A81605FF44051022002F0FB
:105E80000BFC286A18B10B480078042805D1EE6095
:105E90000121002000F04EFA2E70F0BDA403002076
:105EA0009A03002070030020480100206C010020AC
:105EB000E403002098030020F0B5734E0400491C51
:105EC0004F0200F0BDF88021300001F065FD0A208E
:105ED00000F09CF8380CC0B200F098F8380A4A4F2D
:105EE000C0B200F093F8002000F090F85FF48075E5
:105EF00003E014F8010B00F089F82800C51900042C
:105F0000F7D18021300001F045FDBDE8F040A7E069
:105F1000F0B55D4E04005FF480750F0000F090F85E
:105F20008021300001F038FD0A2000F06FF8380CB5
:105F3000C0B200F06BF8380AC0B200F067F8F8B2EF
:105F4000314F01E014F8010B00F060F82800C5198A
:105F50000004F7D18021300001F01CFDBDE8F040C5
:105F60007EE00000F0B5484E040015000F008021CF
:105F7000300001F011FD032000F048F8380CC0B2E9
:105F800000F044F8380AC0B200F040F8F8B21E4FF2
:105F900000F03CF804E0A52000F038F804F8010B0C
:105FA0002800C5190004F6D180213000BDE8F0407A
:105FB00001F0F0BCF0B5344E0400491C4F028021C2
:105FC000300001F0E9FC032000F020F8380CC0B2EA
:105FD00000F01CF8380A0C4FC0B200F017F800208F
:105FE00000F014F85FF4807504E0A52000F00EF8CE
:105FF00004F8010B2800C5190004F6D180213000F7
:10600000BDE8F04001F0C6BCFFFF000030B50B4D0D
:1060100004000221280001F0D1FD0028F9D0210060
:10602000280001F0C7FD0121280001F0C7FD00286C
:10603000F9D0280001F0C0FDC0B230BD003C0040E6
:1060400010B5114C8021200001F0A6FC0620FFF7BE
:10605000DDFF80212000BDE8104001F09BBC000066
:1060600010B5094C8021200001F096FC0520FFF7B7
:10607000CDFFA520FFF7CAFFC007FAD4802120007A
:10608000BDE8104001F086BC000C014004485FF4FC
:1060900080518160C908416009030160704700BFF9
:1060A0006C030020944800B590F82010891E0ED093
:1060B000491E15D0491E01291BD8002100F8201FB8
:1060C0005FF4405102205DF804EB02F0E5BAC17BB9
:1060D00028290ED1816A406A5DF804EB00F034BBD8
:1060E0000121002000F026F95FF44051022002F067
:1060F000D3FA00BD30B5804C0220E57B02F06AFB8C
:10610000608402467D48D82102F090FA94F820007D
:1061100010B1012803D00AE0BDE8304014E02A2D78
:1061200006D1A16A606ABDE8304000F039BB0220A8
:1061300000F022F92421052000F0FCFA00210220C1
:10614000BDE83040F6E0000030B56B4C0021002582
:10615000608C30B103E0694B5B5C6354491C814245
:10616000F9D3844962681F284A60A2688A6005D012
:10617000022000F001F925601A2126E0E27B282A9E
:1061800001D02A2A0FD1607CA17C090451EA006069
:10619000E17C50EA0120217D0143A07D6162E17D27
:1061A00051EA0020A06220685149884240F09B805B
:1061B0005048617B0068884203D3A07B08B1112856
:1061C0000BD3022000F0D8F82421052000F0B2FA09
:1061D0000021012000F0AEF830BD606AA16AAF2A4C
:1061E00000F28180DFE802F06D7F7F58797F7F7F4A
:1061F0007C7F7C7F7F7F7F7F7F7F5B7F7F7C7F7FDC
:106200007F7F615E7F7C5E7F7F7F7F677F6A7F7F2E
:10621000707F737F7F7F7F767F7F7F7F7F7F7F7FB2
:106220007F7F7F7F7F7F7F7F7F7F7F7F7F7F7F7F7E
:106230007F7F7F7F7F7F7F7F7F7F7F7F7F7C7F7F71
:106240007F7F647F7F7F7F7F7F7F7F7F7F7F7F7F79
:106250007F7F7F7F7F7F7F7F7F7F7F7F7F7F7F7F4E
:106260007F7F7F7F7F7F7F7F7F7F7F7F7F7F7F7F3E
:106270007C7F7C7F7F7F7F7C7F7F7F7F7F7F7F7F37
:106280007F7F7F7F7F7F7C7F7F7F7F7F7F7F7F7F21
:106290007C7F7C7F7F7F7F7C00F042FA30BD00F006
:1062A000E5F930BD00F04CFA30BD00F02DFA30BDFC
:1062B00000F030FA30BD00F0EBF930BD00F004FA28
:1062C00030BD00F0B5FA30BD00F03EFA30BD00F050
:1062D00067FA30BD00F092FA30BD00F0B3FA30BD7D
:1062E00000F0B2FA30BD022000F046F820216CE741
:1062F00055534243F403002078030020A4030020F8
:1063000010B50C002200982102F07CF92100012038
:1063100002F038FA3021012002F0ACF904480321E0
:10632000017014488168091B81600021017310BD50
:106330009803002010B502000E480C000B490273B0
:106340000D220160982102F05DF90D21012002F07B
:1063500019FA0748052180F8201034B1042100F80B
:10636000201F3021012002F085F910BD5553425302
:1063700078030020E403002000B520B1012808D0F4
:10638000022809D000BD102101205DF804EB02F0C5
:1063900071B95FF4805105E01021012002F06AF923
:1063A0005FF4805102205DF804EB02F075B9000043
:1063B000FFF778BEFFF79EBE0B4830B50B4C0C4D77
:1063C0000168218021882A880A40510504D509499D
:1063D0000160094800688047208829880140080436
:1063E00048BF01F0E1FF30BD445C0040480400209C
:1063F0004C040020FFFB00005800002010B5FEF701
:106400005FFD8F4800240068847200F01BF9054886
:10641000054904605FF40440088004490860494865
:10642000046010BD445C00404C040020405C00400F
:106430003148324930B5324D097800240470804823
:1064400000684172002002F001F95FF400712046FB
:1064500002F004F92021204602F00CF91821204610
:1064600002F070F995F82C10204602F097F95821A7
:10647000204602F05BF9204602F02EF9204602F099
:106480001FF92146012002F0E9F89821012002F0CD
:106490004DF92021012002F0EDF82146012002F003
:1064A000FBF82146022002F0D9F8D821022002F0A0
:1064B00049F995F82C10022002F070F95FF4405170
:1064C000022002F0E9F82146022002F0D3F815F884
:1064D0002C1F204602F062F9204602F0F1F8204617
:1064E00001F030FF1748012101603A483A49016044
:1064F0003A48047030BD00BF16040020CF95000854
:10650000540000204E4800B50068807A58B10D480C
:1065100005210160012002F0F7F8022002F0E6F800
:106520002E480021017000BD2A482B4900B50068A3
:1065300088421CBF0220FFF71FFF00BD0148042155
:1065400001607047F80300207047000070470000AA
:106550003B4900B509680A785206520E212A0DD12E
:10656000FE280BD1488848B9888838B9C8880128DE
:1065700004D10748020003D1022000BD022000BD63
:1065800088610020488200F04FF8002000BD00BF65
:10659000296600082A4900B509680A785206520E91
:1065A000212A15D1FF2813D1488888B9888878B95D
:1065B000C88868B9012002F0A7F8022002F096F816
:1065C000044805490160054800210170002000BD14
:1065D000022000BD78030020555342439803002059
:1065E00009B10220704700B102207047014901F053
:1065F00045BC00BFA8000020014901F03FBC00BF1E
:10660000B00000200E4900B50968C978062924BFEA
:10661000002000BD034A12EBC1015DF804EB01F05C
:106620002DBC00BFB800002028B905480121006832
:106630000182002070470148704700BFF40300202A
:10664000280400200848074A012101600021016058
:106650001160034A5FF4E05111800160002070472F
:106660004C040020445C0040405C00408249087CAF
:10667000C00702D50448052104E0C97C0348252948
:1066800028BF2421FFF73CBEFC030020E0000020CF
:1066900000B5FFF7FBFC8E4801680A480A0E02713C
:1066A0000A0C42710A0AC1718A49827109680A0C8E
:1066B00042720A0A8272C1720C215DF804EBFFF784
:1066C0001FBE00BF2401002000B5FFF7DFFC80489B
:1066D00001680C484A1E491EC1707E49130E0370A2
:1066E0000968130C4370120A82700A0E02710A0CB8
:1066F00042710A0A8271C17108215DF804EBFFF74B
:10670000FFBD00BF0404002001480421FFF7F8BDCD
:106710000401002001480821FFF7F2BD0801002014
:1067200003480178132928BF12210448FFF7E8BD68
:106730008B030020014A90701173704710010020F4
:1067400001210020FFF7F6BD70B52A4E04000D00B0
:106750003078F0B92A002100282000F08FF8E8B145
:1067600025480078000607D5022030702900200057
:10677000BDE87040FFF7F6BA0220FFF7FDFD2421C7
:106780000520FFF7D7FF01210120BDE87040FFF78A
:10679000D1BD022804BF2046FFF7E4FA70BD000017
:1067A00010B5144C2278FAB90A0001002A2000F032
:1067B00065F8E8B110480078000608D40120207080
:1067C0005FF440510220BDE8104001F065BF002099
:1067D000FFF7D2FD24210520FFF7ACFF00210120A7
:1067E000BDE81040FFF7A6BD012A08BFFFF704FB74
:1067F00010BD000098030020840300201E4800B54F
:10680000816841B9007C400705D4012100205DF872
:1068100004EBFFF78FBD0220FFF7AEFD242105201A
:10682000FFF788FF002101205DF804EBFFF782BD30
:1068300000B5FFF72BFC012100205DF804EBFFF70A
:1068400079BD0000FFF722BC0B4800B5816809B98B
:10685000002005E0007B000601D5002000E00220BA
:10686000FFF78AFD20210520FFF764FF00210120AA
:106870005DF804EBFFF75EBD78030020144B00B514
:1068800089181B688B4209D22A2804BF0220FFF70F
:1068900073FD0020FFF770FD21210EE00D4B0E4926
:1068A0001B6809685A43914210D02A2801D102205E
:1068B00000E00020FFF760FD24210520FFF73AFFEC
:1068C00000210120FFF736FD002000BD012000BDA2
:1068D00074030020700300208003002030BF704745
:1068E00020BF704740BF7047BFF36F8F7047BFF343
:1068F0004F8F7047BFF35F8F704701DF7047EFF333
:106900001480704780F31488BFF36F8F7047EFF3E4
:106910000980704780F309887047EFF3088070475B
:1069200080F30888704762B6704772B67047EFF31D
:106930001080704761B6704771B67047EFF31380EF
:10694000704780F311887047EFF31280704740BAA8
:10695000704700BA7047000000B5080011005FF4EE
:1069600000724902FDF77AFC002000BD30B50C0032
:10697000200055022900FDF76FFC05F2001104F21A
:106980000010FDF769FC002030BD0000F0B51D00CF
:106990000C00160028702E615FF400730020FFF7D2
:1069A000DBFF10B15FF0FF3077E0270017F80B0F27
:1069B000797850EA0120A886B87828753979F8786E
:1069C00050EA0120E882797A387A50EA0120A861F9
:1069D0000AD1B97D787D50EA0120F97D50EA014065
:1069E000397E50EA0160A861397BF87A50EA0120CB
:1069F000E8610ED1B97E787E0B2250EA0120F97E43
:106A000050EA0140397F50EA0160E86121004731D6
:106A100002E00B2221002B31A81C01F033FF0020E3
:106A20006873F979B87950EA01202884A98EEA8A36
:106A3000490AB2184A43AA6258B1EB6940014B4374
:106A400012EB4301021210EBD25011EB60202863CD
:106A50000FE0E869484312EB4000286314F82C0F5C
:106A6000617850EA0120A17850EA0140E17850EACB
:106A70000161E962A869296B401A297DB0FBF1F038
:106A800006496862884201D2002004E00449884235
:106A90002CBF0220012068700020F0BDF50F00001F
:106AA000F5FF00002DE9F04782B014001D0080467C
:106AB00098F801008946D1498A46D0B915EB5506A8
:106AC0005FF400723100684601F0BCFED8F828106F
:106AD000009847182068874214D098F800000123D6
:106AE0003A004946FFF738FF58B100202060504671
:106AF0005DE0012801D16E00E2E70228F7D1AE0087
:106B0000DEE727605FF400723100684601F09AFE0C
:106B100098F80110019E00292FD1974886421DD177
:106B200098F8000099F8FF617F1C01233A0049465C
:106B3000FFF712FF0028D8D12760E80707D599F89A
:106B4000001016F0F000090151EA10162EE099F835
:106B500000000007000F56EA002627E016EB0900A8
:106B6000E9070178407803D5000150EA11161DE0CD
:106B70000007000F51EA002618E016EB0900012972
:106B800004D10178407851EA00260FE002290CD1A7
:106B90004278017851EA02218278C07851EA0241B4
:106BA00051EA00600601360900E05646300002B0A6
:106BB000BDE8F0872DE9F04F83B00C9F04008846B4
:106BC000607815001E00F0B916EB56093F053F0D21
:106BD0005FF40072494601A801F034FEA16A0198F1
:106BE0004018824600208346286882451DD02078C0
:106BF000012352464146FFF7AFFEA0B1C5F800B0F1
:106C00005FF0FF30B5E0012803D170008146BFB2CC
:106C1000DEE7022804D1B00081463F013F09D7E7F3
:106C20005FF0FF30A5E0C5F800A05FF400724946B0
:106C300001A801F007FE029881466078002869D11A
:106C4000F00748BF3F014C4917F47060000A8DF807
:106C5000000017F0F000894547D108F2FF11F20754
:106C600005D50A781207120F1043087000E00F7064
:106C70002A68207801234146FFF778FE38B9286852
:106C8000E1690123421820784146FFF76FFE002892
:106C90006FD15246521C2A60207801234146FFF7EB
:106CA0005BFEF8B9F00703D5380A88F8000008E061
:106CB00098F800009DF8001010F0F000014388F8EB
:106CC00000102A68207801234146FFF74FFE002874
:106CD0004FD12868E1690123421820784146FFF727
:106CE00045FE46E0C5F800B043E019EB0801F207A5
:106CF00007D50A781207120F10430870380A487037
:106D0000DFE70F7048789DF8002010F0F000024394
:106D10004A70D6E73A0A19EB0801012811D10F7021
:106D20004A702A68207801234146FFF71FFE00BB06
:106D30002868E1690123421820784146FFF716FED2
:106D400017E0022813D10F704A70380C8870C87889
:106D500017F07062120E10F0F0000243CA702A6839
:106D6000207801234146FFF701FE10B9B1E75FF03B
:106D7000FF3003B0BDE8F08FFF01000070B50B22BB
:106D800004000D002600202101F088FD0020E072A3
:106D900005E07B2812D2E03006F8010B6D1C287844
:106DA00078B12F280DD0311B0B290ADA6128F0D2D7
:106DB0002E2803D16D1C26000836F0E706F8010BDB
:106DC000ECE7200070BD000070B581B004000D003C
:106DD00000200090022600E0761C606A864209D2FC
:106DE00033006A4629002000FFF75CFE0028F3D13B
:106DF000300000E0014801B070BD0000F7FFFF0F58
:106E0000F0B58BB0040015000F00380001F06AFDEA
:106E1000002638B1380001F065FD01281ED1387810
:106E20002F281BD16078022810D1E06A0123286046
:106E30002E716E71E16A227D206B891E514310EB29
:106E40004102A9682078FFF787FD8CE02E602E7143
:106E50006E71E26AA96820780123F4E7607802285D
:106E600013D1E06A012328602E716E71E16A227DE0
:106E7000206B891E514310EB4102A9682078FFF76F
:106E80006BFD78B15FF0FF306DE02E602E716E719A
:106E9000E26AA96820780123FFF75EFD0028F1D19E
:106EA00000E07F1C38782F28FBD03878002855D098
:106EB000390008A8FFF762FF00208DF800006A463D
:106EC0002900200000F052F830B90B2208A96846CA
:106ED00001F0C6FC0028F2D10B2208A9684601F097
:106EE000BFFC28BB9DF80B00C00621D59DF81B10E8
:106EF0009DF81A0050EA01206178022907D19DF817
:106F0000141050EA01409DF8151050EA0160286005
:106F10002E716E71227D216B801E0123504311EB77
:106F20004002A9682078FFF717FD0028AAD10CE0DD
:106F30000B2208A9684601F093FC30B99DF80B00BC
:106F4000C00602D403200EE07F1C38782F2801D021
:106F50000028F9D12F28A8D17F1CA6E7286800288F
:106F600014BF002003200BB0F0BD0000F0B581B0CD
:106F700004000D0068791700002610283FD36E71B9
:106F80002879401C28712B6873B9228CC0B201018A
:106F9000914201D3012052E0E16A01230A18A96855
:106FA0002078FFF7D9FC4AE0217DC0B288421CD38B
:106FB00024482E71834201D3607850B12249607811
:106FC0008B4201D3012804D054498B4207D30228B5
:106FD00005D1287BC0074CBF052001202FE0A96800
:106FE0006A462000FFF75EFD28602968227D206B3D
:106FF000891E012301FB020029794218CFE7A96805
:10700000202211EB4011380001F03CFC6879401C53
:107010006871387808B1E52805D1287BC00754BFCE
:10702000012000200BE0F97A0907090F0F2901D18F
:107030003E7003E0052804BFE5203870002001B051
:10704000F0BD0000F70F0000F7FF0000F0B581B0C1
:10705000040015001F00FFF7D3FE10B1032001B09C
:10706000F0BD287B50F0010028733A002900200071
:10707000FFF77CFF060003D138780028F5D1EEE752
:10708000012802D15FF0FF30E9E70528FAD1A968AD
:107090002000FFF799FE060020488642F2D0A8683B
:1070A0005FF40072002101F0F9FB002700970EE069
:1070B000226BB31E03FB0020009A01238218207864
:1070C000FFF754FC0028DDD10098401C0090207D83
:1070D000009AA9688242EBD3009740B42B6801AABA
:1070E0002000FFF767FD2E602F7101206871607826
:1070F00001B020B1012804D0022804D0C2E7A24E7A
:1071000002E0A24E00E0A24E200040B42B68A96825
:1071100001AAFFF74FFD01B0B4E70000F7FFFF0F32
:107120002DE9F047A0B0289D0400904699460F0035
:107130001C220021280001F0B1FB85F809804022C3
:10714000390010A801F0D6FB00208DF87F0010A9AF
:10715000380001F0ADFB002630B1042011E110A988
:10716000491C10A801F0B6FB9DF840002F28F6D06E
:1071700010AF380000787F1C0028FAD17F1E10A8BD
:107180008246BA4502D238782F28F7D138782F288E
:1071900008BF7F1C39000DA8FFF7F0FDBA4538BFC6
:1071A0007F1E38782F2802D010A8874200D13E7069
:1071B000CDF808906A4610A92000FFF721FE08B11B
:1071C0000320DEE004AA69462000FFF7CFFE012875
:1071D0000DD140468007F3D504AB6A4610A92000C4
:1071E000FFF734FF002856D05FF0FF30C9E00B22D4
:1071F0000DA904A801F034FB0028E3D19DF81B0081
:10720000C006DDD42C60AE61009818B9E06A9DF824
:1072100004100AE00099227D206B891E5143A28E42
:10722000520A01FB02009DF80410401868609DF8A6
:107230000500401E2872607802280ED19DF82B10A0
:107240009DF82A0050EA01209DF8241050EA0140E0
:107250009DF8251050EA016005E09DF82B109DF87F
:107260002A0050EA01206861E8609DF82D109DF821
:107270002C0050EA01209DF82E1050EA01409DF8A4
:107280002F1050EA01602861687A022804BF0320A9
:107290006872002075E02022002104A801F0FEFAA7
:1072A0000B220DA904A801F0EDFA30468DF81E005E
:1072B0008DF81F008DF820008DF821008DF8260034
:1072C0008DF827008DF828008DF829004946200008
:1072D000FFF77AFD01008DF82A10090A8DF82B10AE
:1072E000010C8DF82410010E8DF825102C60AE6174
:1072F000009919B9E16A9DF8042009E0237D226B09
:10730000891E5943A38E5B0A01FB03219DF80420CB
:107310008A186A609DF805100123491E2972686168
:10732000E8602E6120784946FFF716FB00287FF4BD
:107330005BAF9DF80500202204A919EB401020380E
:1073400001F0A0FA6A68207801234946FFF70EFB96
:1073500000287FF449AF607820B1012804D00228CA
:1073600004D041E7084802E0084800E008480C96CD
:10737000494601B46B690DAA2000FFF71BFC0020F1
:1073800001B020B0BDE8F087F80F0000F8FF000062
:10739000F8FFFF0F2DE9F04F87B0109F04008846DB
:1073A0000393A16900208146206916000025401A38
:1073B000B84238BF0746C3F8009000E00025002F10
:1073C00000F0BD80002D40F0BA802068A169027DE8
:1073D000808E424305A801F027FA06995FF40072F7
:1073E00001A801F021FA22686069116B137D928E69
:1073F000801E5843520A00FB021001995FF400728C
:107400004518A16901A801F00FFAF019049002983B
:10741000002830D0206801232A0000784146FFF779
:107420009BFAA16905005FF4007201A801F0FCF964
:107430000298D0F5007080B2824683465F4513D330
:10744000524641424046401800F20021300001F00F
:1074500019FA5046CDF800B03618A0695946B7EB76
:107460000B074018A0612FE03A0041424046401807
:1074700000F200211FE02068B7F5007F12D301233E
:1074800000782A003100FFF767FA05002E4806F25F
:1074900000263F18A06900F20020A0615FF4007090
:1074A000009011E0012300782A004146FFF754FACA
:1074B00005003A004146300001F0E4F9A069049E5D
:1074C000C019A061009700270398009A01688918E5
:1074D000016020680099027D808E4243A069411AB4
:1074E00001A801F0A1F92068A169027D808E4243C4
:1074F00005A801F099F90198059988423FF45FAF1A
:10750000CDF800902068417821B961690F4A914215
:10751000BFF454AF41786369012903D10C498B4210
:10752000BFF44CAF4178022903D10A498B42BFF422
:1075300045AF6A464146FFF7B5FA60613FE728006C
:1075400007B0BDE8F08F000000FEFFFFF80F00005D
:10755000F8FF0000F8FFFF0F2DE9F04F89B0129FF0
:107560000400049300208146607A884616000025B6
:10757000022802D25FF0FF305EE1C3F8009077E0AE
:107580003A0031004346181801F07CF93DB92068F3
:107590000123524600784146FFF7E8F90500A0694B
:1075A000059EC019A0612169814238BF2061009702
:1075B0000027C1E02068B7F5007F16D301230078CB
:1075C00052463100FFF7D2F905009D4806F2002629
:1075D0003F18A06900F20020A0612169814238BFF4
:1075E00020615FF400700090A6E0A16922699142D9
:1075F00012D20078012352464146FFF7ADF905004B
:1076000011D13A003100404601F03CF920680123D5
:1076100052460078414603E000780123524631008B
:10762000FFF7A4F90500A069059EC019A0612169B2
:107630008142BCD22061BAE720B4099B206801AA2C
:107640004146FFF7B7FA65612068417801B031B172
:10765000012900F0BB80022900F0BA80BAE0794D20
:10766000414620B4636901AA0025FFF7A3FA01B0DF
:107670002068002F00F0B380002D40F0B080027D24
:10768000808EA169424306A801F0CEF807995FF405
:10769000007202A801F0C8F822686069116B137DBE
:1076A000928E801E5843520A00FB021002995FF42A
:1076B00000724018A169824602A801F0B5F8F019DD
:1076C0000590039800283FF475AF206801235246C7
:1076D00000784146FFF740F9A16905005FF40072A8
:1076E00002A801F0A1F8039880B20190D0F5007BC8
:1076F0005F45FFF445AF5A4631004346181801F084
:10770000C1F83DB920680123524600784146FFF791
:107710002DF90500CDF800B0019880B241427018F3
:1077200000F20026A0691BEB0000A06121698142E4
:1077300038BF2061B7EB0B070498009A01688918DD
:10774000016020680099027D808E4243A069411A41
:1077500002A801F069F82068A169027D808E424389
:1077600006A801F061F80298069988423FF480AFBC
:10777000CDF8009063696A46414608932068FFF798
:1077800091F96061607A02287FF472AF20686169C4
:10779000427812B92B4A91420BD24278012A02D187
:1077A0002A4A914205D24278022A16D1284A9142A9
:1077B00013D34146FFF708FB05002348CDF800909E
:1077C00085427FF439AF5FF0FF3035E01F4D47E76A
:1077D0001F4D45E75FF0FF302EE0002548E7626867
:1077E000007801234146FFF7B7F810B15FF0FF3092
:1077F00022E0207A2169012318EB40100177207ADA
:10780000216918EB4010090A4177207A216918EBA9
:107810004010090C8177207A216918EB4010090E7D
:10782000C1772068626841460078FFF79FF810B181
:107830005FF0FF3000E0280009B0BDE8F08F0000E5
:1078400000FEFFFFF80F0000F7FFFF0FF8FF00003A
:10785000F8FFFF0F09490A6812F038020A600A6847
:107860001043086070470000044910230A689A43D7
:107870000A600A6810430860704700000020024058
:1078800002482549016025490160704704200240F3
:107890002348016851F080010160704770B51D4DAB
:1078A0000400280000F056F8042813D11C4E30685C
:1078B00050F00200306008480460306850F040002A
:1078C0003060280000F046F8012803D03168034AF0
:1078D0000A40326070BD00BF14200240FD1F00004E
:1078E00070B504000F200D0000F034F804280ED10C
:1078F0000B4E306850F00100306025800F2000F002
:1079000029F8012803D03168014A0A40326070BD6D
:10791000FE1F0000FF0F000023016745AB89EFCD7C
:10792000102002400A4908607047000008480168BA
:10793000C90744BF012070470168490744BF0220BE
:1079400070470068C00644BF03207047042070479A
:107950000C20024010B50400FFF7E8FF04E000F03F
:107960000BF8FFF7E3FF641E012801D1002CF6D1CC
:1079700004B9052010BD000081B000200090FF2058
:1079800001E00098401E009000980028F9D101B055
:107990007047000001617047416170472949024A00
:1079A00002430A60704700000000FA050100F0B4CD
:1079B0000A78C87858B323481B4C9310006814EB1E
:1079C0008305AC462C684F7810F4E060D0F5E06099
:1079D000000A0426351A8E789207D20EFF239340B0
:1079E000AF403D000F27C74037402F43380190403C
:1079F0000C4A65469C43034023432B6008780123CF
:107A00004111C006C00E834042F8213007E007490B
:107A100050110123D206D20E934041F82030F0BC21
:107A2000704700BF00E100E000E400E080E100E01A
:107A3000034A024B0B4003431360704780FFFF1F54
:107A400008ED00E00CED00E043480D4B016851F0FB
:107A50000101016034490A6813400B600268094B58
:107A60001340036002687FF48023134003600868BA
:107A70007FF4FE0202403B480A600021016070472B
:107A80000000FFF8FFFFF6FE33497FF480330A68F9
:107A900013400B600A687FF4802313400B605FF48F
:107AA0008032904203D09200904205D0704708681F
:107AB00050F4803008607047086850F4A0200860D7
:107AC0007047000010B581B000240094312000F010
:107AD0002DF80099491C009118B90098B0F5A06FD5
:107AE000F4D1312000F022F800B10124200001B0CF
:107AF00010BD000001490860704700BF60004242AD
:107B0000094903230A689A4310430860704700003C
:107B10000548006810F00C0070470000014908603B
:107B2000704700BFD80042420410024041090129B9
:107B300002D10949096805E0022919BF0849096805
:107B4000064909680122C006C00E82400A401CBFD7
:107B500001207047002070470010024020100240B2
:107B6000241002400810024002880B8812F441528F
:107B700013434A881A438B881343CA881A430B89D4
:107B800013434A891A438B891343CA891A430280D3
:107B9000098A0182704700000029018803D051F052
:107BA000400101807047024A0A400280704700BFCE
:107BB000BFFF0000818170478089704700B5008950
:107BC00008421CBF012000BD002000BD10B5B14C13
:107BD00020B9012120680182002010BDA64800685C
:107BE0000068804720680A3010BD0000A9480A4A92
:107BF00000B500681278C1788A420AD3827842B907
:107C0000828832B981729C480068406880470020B1
:107C100000BD022000BD00BF3101002010B59D4C09
:107C200020B9012120680182002010BD924800681F
:107C30008068804720680C3010BD00000F4A10B5E6
:107C4000944C126820689269C17840799047216805
:107C50008A7A22B118B9087908B9887808B102205F
:107C600010BD85480068C068804720684179C172AE
:107C70002068C1780173002010BD00002C04002092
:107C8000844910B5096818B902200882002010BD87
:107C9000204C002020800878420615D1487A8106C1
:107CA00003D5217851F0020121704006207808D5D3
:107CB00010F0FE00207070480068006980472000C6
:107CC00010BD50F00100F5E74206520E012A04BF34
:107CD000204610BD4006400E022818D14979207870
:107CE0000A07120F50F00100090607D5594951F84B
:107CF000221011F030011029DDD1DBE7554951F890
:107D0000221011F44051B1F5805FD4D1D2E70020A8
:107D100010BD00BF4A0400205E4870B500680178BD
:107D20004906490E05D1417A11F0DF014172002068
:107D300070BD022903D1418809B9017909B1022036
:107D400070BD417980220C0094430A0605D5414A52
:107D500052F8242012F0300204E03E4A52F8242067
:107D600012F440523A4B1B789C42E8D2002AE6D0EB
:107D7000807A0028E3D0374810EB8405080628688D
:107D80000BD510F03000102822D1200000F0BCFCF0
:107D90003021200000F06EFC1AE010F44050B0F5E5
:107DA000805F15D12C4E5CB90C480178002000F0A2
:107DB000F5FC284801680E4096F44051016007E048
:107DC000200000F093FC2868064096F4405028609C
:107DD0002948006840698047002070BD800000206D
:107DE0002C4810B580230168487902009A430306A5
:107DF00005D5184B53F8223013F0300304E0154B2F
:107E000053F8223013F44053114C2478A24204D288
:107E10004C8814B90BB1897A09B9022010BD0D49FB
:107E200011EB82010A68000604D50848104090F062
:107E3000100003E00848104090F4805008600E489D
:107E4000006880698047002010BD00BFBF8F000020
:107E500030010020005C00408FBF00000D4800B5DD
:107E60000068417A51F02001417203480068C069FE
:107E70008047002000BD000030040020054A126841
:107E8000538A20B98888C01A108200207047086879
:107E9000C018704728040020F0B5734C256835F8E9
:107EA000100FA9680A0015D0A0B1AE88B04238BF43
:107EB00006463000884707002888801B288068888D
:107EC00080196880002000F053FC32000100380067
:107ED00000F0ACFB674E2888302738B133483902B0
:107EE00001800021002000F04DFC37802988AA88FD
:107EF0002068914222BF03210172F0BD11B105211A
:107F00000172F0BD062101725848594900220068EB
:107F100080B241F810203780F0BD000052482DE9B2
:107F2000F04104248046D8F80000050035F8101F01
:107F300099B9007A042810D1B1480178012909D1F2
:107F40004A4A4B4B0021126892B243F81210302279
:107F5000017022E0072410221FE0AE888E4223D356
:107F6000B14238BF0E46A96830008847070000209C
:107F700000F0F4FB32000100380000F043FB310058
:107F8000002000F0FFFB288830221102801B28808F
:107F90006888801968800548018036480280D8F8D2
:107FA00000000472BDE8F0810224DCE74E040020EA
:107FB00070B52D4D08242868017846784A0628D1E6
:107FC000092E02D1FFF712FE34E08188C278052E17
:107FD0000AD1802A44D28278002A41D100293FD197
:107FE000807A002831D03BE0407A032E07D1012A65
:107FF00021D101BB80061ED5FFF730FF1AE0012E0C
:1080000019D1012A17D1B1B9800614D5FFF784FE22
:1080100010E04806400E012804D10B2E0BD1FFF7CB
:108020000DFE07E0022806D1012EEFD0032E02D16B
:10803000FFF7D6FE40B1BE4930000968496988475C
:10804000032801D109240BE050B90848084900224F
:108050000068062480B241F81020064830210180D3
:108060002868047270BD000028040020505C0040A5
:108070000460004050040020AD4A2DE9F043AE4DAD
:1080800081B009262868447803789046D8F8002003
:108090005906490EB146062C0ED100296AD18078C6
:1080A000012801D1D46954E0022801D1146A50E0BA
:1080B00003285FD1546A4CE09269C6884788002C37
:1080C00033D1002F56D1022E54D10479002C51D136
:1080D000474C11B9818800293BD040795906490E97
:1080E000012908D100219047002843D12868807ACF
:1080F00000283FD02DE002293CD10107090F10F0E4
:108100007002000605D59E4850F8210010F030009E
:1081100004E09B4850F8210010F44050974B1B7826
:10812000994227D232BB28B313E0082C02D109BBF5
:10813000304C0EE00A2C1DD101291BD1817AC9B126
:10814000C7B90179B1B9012E14D14079904788B9E6
:10815000294C20000ED02868002141828461002033
:10816000A04700212A68254B108A98420FD182F837
:10817000089039E02868D8F80010407809698847E5
:1081800001000328EED1286880F808902CE002292D
:1081900000D010B90820107226E0117809061DD50C
:1081A000D1880091D8F80030009C844202D2009817
:1081B00010820DE088420BD293F82C10104C8842AC
:1081C00001D2002003E000F0B3FB08B901202070C9
:1081D00013F82C0F9082FFF7A1FE05E00320107228
:1081E00056485FF44051018001B0BDE8F08300BF04
:1081F000817C0008CD7B00081D7C0008FFFF00008B
:10820000530400201C491A4A1A4830B509684A4CE0
:1082100089B252F8111089B210EB41052068017A39
:10822000092917D02978017020686978AD1CAD1C28
:10823000417028000088AD1CAD1C00F0E1FA2168F7
:10824000488028000088AD1C00F0DAFA2168888098
:108250006888C8802068012101722068C08810B930
:10826000FFF7A6FE01E0FFF707FF00F047F830BD7B
:108270000860004000600040505C004030B52E4C6B
:108280002068017A022901D0042904D1FFF746FEB3
:108290002068057A13E00825062910D141780529C0
:1082A00009D10178490606D1C07800F04BF806489C
:1082B0000068006A80471E48006880688047206820
:1082C0000572BDE8304019E03004002030B51A4C8A
:1082D0002068007A032801D0052804D1FFF7DCFDCF
:1082E0002068057A06E00825072803D110480068B1
:1082F000C068804720680572BDE830400D4800B571
:108300000178002000F04AFA0B480068017A082939
:1083100006D10A495FF480520A80094910220A8076
:10832000007A092804BF012000BD002000BD000024
:108330002C04002080000020280400204E0400208F
:10834000500400200D4970B40022097851B90BE0A7
:108350000B4C084ED3B2521C14EB830425682E40FC
:10836000334323608A42F3D3034950F0800008600E
:1083700070BC70478F8F00004C5C004030010020C3
:10838000005C0040704700000448054A0221017269
:108390000449C06142620162086800470C04002081
:1083A00084000020540000208D482DE9F04F924DAC
:1083B000714E80468B4881461DE015EB810217689F
:1083C000BFB23B0408D5136818401060874810EB13
:1083D0008100001F0068804738060CD5207815EB17
:1083E00080010A681AEA02020A60854911EB8000DE
:1083F000001F00688047D9F80000A8F800000004BA
:1084000040F1B8807A487B4CC9F80000B8F8000009
:1084100001077A48090F2170824673480029CCD1A0
:108420005649574C8B46296811F44051ABF800105F
:10843000296811F03001ABF802102968214091F44D
:10844000005129602968314091F020012960B8F875
:108450000010C90621D428681AEA00002860FFF736
:108460000DFF28680440BBF80000C10448BF94F425
:108470008054800402D594F40054A4B22C6028687F
:108480000640BBF80200C10648BF96F01006800601
:108490006FD596F02006B6B26BE02F68BFB23906F2
:1084A00021D528681AEA00002860FFF7E7FE28684F
:1084B0000440BBF80000C10448BF94F48054800419
:1084C00002D594F40054A4B22C6028680640BBF88E
:1084D0000200C10648BF96F01006800649D596F006
:1084E0002006B6B245E0390520D529680840286045
:1084F000FFF788FE28680440BBF80000C10448BFAD
:1085000094F48054800402D594F40054A4B22C60F6
:1085100028680640BBF80200C10648BF96F0100666
:10852000800626D596F02006B6B222E039047FF503
:1085300062AF296808402860FFF7C8FE2868044039
:10854000BBF80000C10448BF94F48054800402D5F5
:1085500094F40054A4B22C6028680640BBF80200D2
:10856000C10648BF96F01006800602D596F0200698
:10857000B6B22E60BDE8F08FBF8F00004E04002021
:108580008FBF000030B5164C164D09E00A68164B37
:1085900013400B60154911EB8000001F00688047F5
:1085A0002868208000041AD51148124928602088C4
:1085B0000007000F0870104911EB80010A6892B2A1
:1085C0001304E3D41206EBD50A680C4B13400B607E
:1085D0000B4911EB8000001F00688047E0E730BDC9
:1085E00048040020445C00408F0F00003800002049
:1085F000FF7F000054040020005C00400F8F00004B
:108600001C000020104B10B4521C13EB41015210FF
:1086100009D044780378801C53EA042321F8023BF4
:10862000891C521EF5D110BC70470000064B521C2D
:1086300013EB4101521005D051F8043B521E20F8B3
:10864000023BF9D170470000006000405249024AE5
:1086500002400A60704700BFF8FF0000324A044B36
:1086600012EB80000268134019430160704700BF9D
:108670008F8900002C4A12EB8000104A03681A40D0
:10868000CB0648BF92F01002890602D592F0200274
:1086900092B2026070470000234A12EB80000D4A3C
:1086A00003681A40CB0448BF92F48052890402D573
:1086B00092F4005292B2026070470000BF8F000037
:1086C000194911EB800003490268114091F44051AF
:1086D000016070478FBF00001349034A11EB80000F
:1086E00001680A40026070478F8E00000E4911EB4E
:1086F00080000168490405D501680A4A0A4052F41D
:108700008041016070470000074911EB800001685B
:10871000490605D50168034A0A4052F0400101604C
:10872000704700008F8F0000005C00401A4A490823
:108730004900126892B212EBC0002C4A42F81010A5
:1087400070470000144A49084900126892B212EBBF
:10875000C000274A42F81010704700000E4909680F
:1087600089B211EBC000214951F8100080B2704766
:108770000949096889B211EBC0001D4951F8100080
:1087800080B27047044A126892B212EBC0001B4AD2
:1087900042F8101070470000505C0040154A126803
:1087A00092B212EBC000144A12EB40003F2908D3EA
:1087B0004A09C90604BF521E92B2910251F4004107
:1087C00005E04A08C90744BF521C92B291020160F9
:1087D000704700000749096889B211EBC0000649DB
:1087E00051F810008005800D7047000000600040C7
:1087F00008600040505C00400C6000400460004095
:108800000106090C51EA1020704700007047000073
:1088100010B581B00400009469460120FFF7F6FF0F
:10882000F9E7000000F078B882B091FBF2F3009312
:1088300002FB13110191DDE90023C0E9002306BC0E
:108840007047000082B091FBF2F3009302FB13111A
:108850000191DDE90023C0E9002306BC7047000058
:1088600010B502E0401C491C521E4AB103780C7836
:10887000A342F7D002D25FF0FF3010BD012010BD3F
:10888000002010BD10B50300002A04E011F8014BD0
:10889000521E03F8014BF9D110BD0000C9B203000C
:1088A000002A02E003F8011B521EFBD170470000B2
:1088B00001E0401C491C02780B789A4203D1002A3F
:1088C000F7D10020704702D25FF0FF3070470120DF
:1088D00070470000020011F8013B02F8013B002B39
:1088E000F9D17047010000E0491C0A78002AFBD149
:1088F000081A704710B5030005E00C7834B1491C24
:10890000521E03F8014B002AF7D122B1002103F8CF
:10891000011B521EF9E710BD014CA646204700007E
:10892000118800088C46B0FBF1F10CFB1100704778
:108930008C4690FBF1F10CFB110070472103000005
:10894000340100203401002032010000000000202A
:10895000548900081A03530054004D0033003200BC
:1089600031003000000000000000000000000000A6
:10897000B1630008858300088583000885830008AB
:1089800085830008858300088583000885830008A7
:10899000B563000885830008858300088583000887
:1089A0008583000885830008FD63000831640008A2
:1089B000496500084D650008516500089565000887
:1089C000E1650008ED650008F96500080566000826
:1089D00000000000400000008583000805650008D5
:1089E00085830008858300088583000829650008C1
:1089F00085830008858300083D650008B49500085C
:108A000012000000C895000820000000E89500084A
:108A100004000000EC9500082600000014960008F1
:108A200026000000000000201A0000003C9600080C
:108A30001000000000800202200000004D696E69F5
:108A40005F44534F466C617368204469736B202008
:108A5000202020202000000003000000000600006D
:108A600000000000700000000000000A000000008C
:108A700000000000000000000000000800000000EE
:068A8000020000000301EA
:108A880048617264776172652056657220322E36AD
:108A980030200000332E3130000000009001F0003B
:108AA800070015000F00C8000010010001011100A7
:108AB800000000040000000435306D56000000007E
:108AC8000000000400000004D0070000302E3156DA
:108AD800000000000000000400000004A00F0000D7
:108AE800302E325600000000FEFF0004FAFF00049A
:108AF800401F0000302E355600000000FFFF000424
:108B0800FAFF0004204E000020315620000000002B
:108B180000000004FAFF0004409C000020325620A8
:108B280000000000FEFF0004FAFF00048038010086
:108B38002035562000000000FFFF0004FAFF000463
:108B4800400D0300213130562100000000000004D0
:108B5800FAFF0004801A0600000000000000000070
:108B68000000000000000000000000002120315338
:108B780020210000E7035F09B004000455A0FC01B0
:108B88003530306D53000000E703AF04580200048D
:108B98002B50FE003230306D53000000E703DF0138
:108BA800F0000004ABB965003130306D53000000AF
:108BB800E703EF0078000004D5DC32002135306D82
:108BC80053210000E70377003C0000046B6E190096
:108BD8002132306D532100006300DF01F0000004F2
:108BE8002B2C0A002131306D532100006300EF0067
:108BF800780000041516050020356D53200000008C
:108C0800630077003C0000040B8B020020326D5398
:108C1800200000000900DF01F00000046B040100DF
:108C280020316D53200000000900EF007800000497
:108C38003582000035303075530000000900770098
:108C48003C0000041B410000323030755300000026
:108C58000000DF01F00000040B1A0000313030750D
:108C6800530000000000EF0078000004050D00002C
:108C78002135307553210000000077003C000004C6
:108C880083060000213230755321000000002F00B8
:108C9800180000049B0200002131307553210000A8
:108CA800000017000C0000044D010000203575532A
:108CB8002000000000000B0006000004A7000000D0
:108CC8002032755320000000000004000300D70381
:108CD800430000002031755320000000000002000E
:108CE8000200330321000000302E357553000000C8
:108CF800000001000100660211000000302E3275EC
:108D080053000000000000000100EC010700000013
:108D1800302E317553000000000000000100F600FD
:108D280003000000203275532B00000000000900EA
:108D38000300D70343000000203175532B000000C7
:108D4800000004000200D703210000002E357553EF
:108D58002B00000000000200010033031100000096
:108D68002E3275532B000000000001000100D703CC
:108D7800070000002E3175532B0000000000000092
:108D88000100EB01030000003C56740000000000E5
:108D980000003C5674000000000001023C567400BC
:108DA8000000000002043C567400000000000306A6
:108DB8003E5674000000000000013E56740000009A
:108DC800000001033E5674000000000002053E56F4
:108DD80074000000000003073A215C210000000035
:108DE80000083A215C2100000000010A3A215C21B8
:108DF80000000000020C3A215C2100000000030E74
:108E08003A215E210000000000093A215E2100009D
:108E18000000010B3A215E2100000000020D3A21FA
:108E28005E2100000000030F3C544C0000000000CD
:108E380000103C544C000000000001123C544C004F
:108E48000000000002143C544C000000000003160F
:108E58003E544C000000000000113E544C0000003D
:108E6800000001133E544C000000000002153E545F
:108E78004C000000000003173C54480000000000AC
:108E880000183C54480000000000011A3C544800F7
:108E980000000000021C3C54480000000000031EB3
:108EA8003E5448000000000000193E5448000000ED
:108EB8000000011B3E54480000000000021D3E5403
:108EC800480000000000031F0000000000001C0014
:108ED80020004000400040004000400020001C00EE
:108EE800000000000000000000000000000000E09A
:108EF8000010000800080008300C600CC000800159
:108F080000033006300C000000080008001000E0E4
:108F18000000000000000000102010201020102089
:108F280010201020F03F000000000000C00FE01FDC
:108F38003030102000000000000000001020303009
:108F4800E01FC00F000000000000C018800D0007DF
:108F58000007800DC0180000000000010001C007D4
:108F6800C007000100010000000000000000FCFF35
:108F780000000000000000000000000100010001E6
:108F880000010001000100000000000000003000A6
:108F9800300000000000000030006000C0008001C8
:108FA80000030006000C0000E01FF03F9020102393
:108FB8001024F03FE01F0000000010081018F03FD8
:108FC800F03F1000100000007010F03090211023C6
:108FD80010263038301800002010303010221022AF
:108FE8001022F03FE01D000000030007000D1019DB
:108FF800F03FF03F10010000203E303E10221022CA
:109008001023F023E0210000E00FF01F103210229F
:109018001022F003E001000000300030F020F021C1
:109028000023003E003C0000E01DF03F102210220B
:109038001022F03FE01D0000001C103E10221022FC
:109048003022E03FC01F0000000000000000600C5C
:10905800600C00000000000040004000400040009C
:109068004000400040004000000000018003C006AE
:10907800600C301810100000000090009000900064
:109088009000900090000000400240024002400220
:109098004002400240020000000010103018600C2E
:1090A800C006800300010000C00F20109027902404
:1090B800D0275010800F0000F007F00F0019003182
:1090C8000019F00FF00700001020F03FF03F1022C9
:1090D8001022F03FE01D0000C00FE01F30301020CC
:1090E80010203030601800001020F03FF03F1020B2
:1090F8003030E01FC00F00001020F03FF03F10227A
:1091080010273030703800001020F03FF03F102258
:109118000027003000380000C00FE01F3030102159
:109128001021E031F0190000F03FF03F000200028A
:109138000002F03FF03F0000000000001020F03F68
:10914800F03F102000000000E000F00010001020A8
:10915800F03FE03F002000001020F03FF03F000308
:10916800000FF03C703000001020F03FF03F10205E
:109178001000300030000000F03FF03F001C000EEF
:10918800001CF03FF03F0000F03FF03F001C000ED5
:109198000007F03FF03F0000C00FE01F3030102004
:1091A8003030E01FC00F00001020F03FF03F1022C9
:1091B8000022003E001C0000E01FF03F102070203D
:1091C8003020F83FE81F00001020F03FF03F002259
:1091D8000023F03FF01C00006018703C102610229D
:1091E8001023F039E0180000000000381030F03F7C
:1091F800F03F103000380000E03FF03F1000100052
:109208001000F03FE03F0000803FC03F60003000AA
:109218006000C03F803F0000C03FF03F7000C001C9
:109228007000F03FC03F00003030F03CC00F00033A
:10923800C00FF03C303000000000003C103EF0034E
:10924800F003103E003C00007038F03090211023ED
:109258001026303C7038000010003000500090019B
:109268001003100CF03F0000000800080008000878
:1092780000080008000800080000000000007CFC4E
:10928800800280020001000100020004000CF01FAF
:10929800F03F000C0004000200018000C000E03F25
:1092A800F03FC00080000001102010201020102086
:1092B8001020102010201020E000F00510051005E7
:1092C800E007F003100000001020F03FE03F10021C
:1092D8001002F003E0010000E003F007100410049E
:1092E8001004300620020000E001F00310061024EC
:1092F800F03FF03F10000000E003F00710051005F4
:10930800100530072003000000001002F01FF03F96
:109318001022003000180000C803EC0724042404BD
:10932800FC03F807000400001020F03FF03F200283
:109338000004F007F0030000000000001004F037FC
:10934800F037100000000000000018001C000404A2
:10935800FC37F837000400001020F03FF03F802170
:10936800C003700630040000000000001020F03F29
:10937800F03F100000000000F007F0070006F003BF
:109388000006F007F00700000004F007F0030004EF
:109398000004F007F0030000E003F00710041004D5
:1093A8001004F007E00300000404FC07FC03440475
:1093B8004004C007800300008003C0074004440441
:1093C800FC07FC03040400001004F007F003100677
:1093D800000400060003000000002002300790058A
:1093E8009004F0066002000000040004E01FF03F53
:1093F8001004300420000000E007F00710001000FF
:10940800E007F007100000000000C007E007300088
:109418003000E007C0070000E007F0073000E00078
:109428003000F007E007000010043006E003C00138
:10943800E0033006100400008007C407440044001D
:109448004400F807F007000030067006D0049005C5
:10945800100730063004000080078004F03C10201C
:10946800D02FD02FD02FD02FD02FD02FD02FD02FFC
:10947800D02FD02FD02FD02FD02FD02FD02FD02FEC
:10948800D02F1020F03F000080078004F03C10200F
:1094980010201020102010204861726477617265D6
:1094A800205665722000000053657269616C204E79
:1094B8006F3A200020202020204453323033204DA2
:1094C800696E692044534F205359532056657220C2
:1094D800202020202020202020202000506C6561A2
:1094E800736520696E707574206D61737465722080
:1094F8006C6963656E63653A2030303030303030E7
:109508003000000020202020202020204C696365A6
:109518006E636520696E707574206572726F722053
:109528002020202020202020200000002020202093
:1095380020202020204C6963656E6365207772695E
:1095480074656E206F6B2020202020202020202092
:109558002000000020202020202020204C69636566
:109568006E63652077726974656E206572726F72BA
:109578002020202020202020200000002020202043
:1095880020205075736820616E79206B657920748E
:109598006F206E65787420737465702020202020F9
:1095A80020000000312E34310000000012010002BA
:1095B800000000408304205700020102030100005C
:1095C80009022000010100C0320904000002080657
:1095D8005004070581024000000705020240000010
:1095E800040309042603530054004D006900630076
:1095F80072006F0065006C00650063007400720003
:109608006F006E00690063007300000026035300BA
:1096180054004D003300320020004D0061007300FB
:1096280073002000530074006F007200610067002F
:109638006500000010035300540020004D00610035
:0696480073007300300006
:040000050800416549
:00000001FF
